:100000000AC02EC01895189518951895189518952A
:100010001895189518958FED8DBFC0ECE0EC4E2E1D
:10002000DD275D2EEEE7F0E0A0E6B0E088278D93B7
:100030003197E9F766248FE087BB8BEF81BB80E7C0
:1000400088BB84E082BB78948BB780648BBFC398F5
:10005000C298C198C09885B7806385BF8895F7CF4F
:10006000F894E2E3F0E0ACE691E097D300916C0005
:100070000E3C08F004C085B7806385BF8895C39A9D
:10008000C29AC19AC09A80E080936A0080E080930F
:100090006900ADE657D3A1E657D380E080936500B1
:1000A000ADE6E5D2C39AC0988CE080936000BC981E
:1000B000AFE69C9197FF04C0B49B0EC09F779C93C2
:1000C000B4990AC088E29F9399272DD39F91B49940
:1000D00003C090689C931ED18AE080936000BD9815
:1000E000AFE69C9196FF04C0B59B0EC09F7B9C938E
:1000F000B5990AC088E29F93992715D39F91B59926
:1001000003C090649C9306D18BE080936000BE98FE
:10011000AFE69C9195FF04C0B69B0EC09F7D9C935B
:10012000B6990AC088E29F939927FDD29F91B6990C
:1001300003C090629C93EED0C09AC19889E08093EE
:100140006000BC98AFE69C9197FF04C0B49B0EC0C2
:100150009F779C93B4990AC088E29F939927E3D232
:100160009F91B49903C090689C93D4D088E0809309
:100170006000BD98AFE69C9196FF04C0B59B0EC091
:100180009F7B9C93B5990AC088E29F939927CBD215
:100190009F91B59903C090649C93BCD087E08093F5
:1001A0006000BE98AFE69C9195FF04C0B69B0EC060
:1001B0009F7D9C93B6990AC088E29F939927B3D2FA
:1001C0009F91B69903C090629C93A4D0C19AC298A3
:1001D00086E080936000BC98AFE69C9197FF04C0D6
:1001E000B49B0EC09F779C93B4990AC088E29F93FA
:1001F000992799D29F91B49903C090689C938AD013
:1002000085E080936000BD98AFE69C9196FF04C0A6
:10021000B59B0EC09F7B9C93B5990AC088E29F93C3
:10022000992781D29F91B59903C090649C9372D015
:1002300084E080936000BE98AFE69C9195FF04C077
:10024000B69B0EC09F7D9C93B6990AC088E29F938F
:10025000992769D29F91B69903C090629C935AD016
:10026000C29AC39883E080936000BC98AFE69C91EB
:1002700097FF04C0B49B0EC09F779C93B4990AC0AB
:1002800088E29F9399274FD29F91B49903C09068B9
:100290009C9340D082E080936000BD98AFE69C9133
:1002A00096FF04C0B59B0EC09F7B9C93B5990AC076
:1002B00088E29F93992737D29F91B59903C09064A4
:1002C0009C9328D081E080936000BE98AFE69C911B
:1002D00095FF04C0B69B0EC09F7D9C93B6990AC043
:1002E00088E29F9399271FD29F91B69903C090628D
:1002F0009C9310D081E090E016D2ADE60D911C9158
:10030000083853E1150710F009F001C0C9CE789400
:1003100018950895ADE616D2939A84E690E003D23C
:1003200093988EE190E0FFD1BF98AFE69C9194FF47
:1003300004C0B7990EC09F7E9C93B79B0AC088E209
:100340009F939927F0D19F91B79B03C090619C9395
:1003500052D1A6E30C9104FB81E00EF480E08F9370
:10036000A6E30C9105FB81E00EF480E09F91892BC0
:100370008F93A6E30C9106FB81E00EF480E09F9141
:10038000892B882309F401C0E4CF00916900013072
:1003900009F00DC08091600080936A00A9E68C91FD
:1003A0008F5F8C9380E080936500D7D00895009193
:1003B0006900023009F001C04DC0009169000330AE
:1003C00009F001C066C0009160000B3009F008C060
:1003D000A9E68C918F5F8C9380E0809365000895EF
:1003E000009160000C3009F034C046E65BE260E04A
:1003F00070E0A1E60D911D912D913C91B0D109F0D5
:1004000001C08EC081E080936600009166000830D4
:1004100010F009F01DC0E6E6F0E0A190EEEFFFEF6E
:10042000AA0CBB1CAA0CBB1CEA0DFB1DA4E194E0AA
:10043000B4D1A1E60D911D912D913C9190D109F07F
:1004400001C0B2C0A6E68C918F5F8C9308F4DDCF1B
:1004500067C03AC0009160000C3009F019C0E2E0BA
:10046000F0E0A4E194E099D1A1E60D911D912D91C8
:100470003C9175D109F401C053C06FD0A1E664D19D
:1004800080E080936500A9E68C918F5F8C9308953E
:100490001BC0009160000C3009F016C0EAE6F0E0E5
:1004A000A190EEEFFFEFAA0CBB1CAA0CBB1CEA0D3F
:1004B000FB1DA1E694E07BE75FD14FD08CEE93E18A
:1004C000ADE68D939C930895A5E68C918F5F8C93F8
:1004D00000916500063010F009F001C001C020C095
:1004E000A1E60D911D912D913C914AE050E060E014
:1004F00070E0CAD0A1E60D931D932D933D93A1E624
:100500000D911D912D913C91A0E64C9155276627A8
:10051000772720D1A1E60D931D932D933D93089548
:10052000ABE68C918F5F8C9389E0809367008FE5B9
:10053000809368001AD000916B00033009F007C067
:10054000ECE3F0E09BD080E080936B0006D08CEE73
:1005500093E1ADE68D939C93089582E080936700CC
:1005600088EC8093680001D0089584E690E0DBD0A9
:1005700081E0809366004091670000916600041757
:1005800010F009F010C0939AA8E68C919927CBD06F
:100590009398A8E68C919927C6D0A6E68C918F5F98
:1005A0008C9308F4E8CF089580E080936B00A1E677
:1005B000CBD0D3DFE2E2F0E0A8E6ECD084EF91E02C
:1005C000B2D0949AA8E6EC91FF2758D09498E1E035
:1005D000F0E054D080916C00815080936C00E2E395
:1005E000F0E0ACE691E07BE7C7D08CEE93E1ADE6BE
:1005F0008D939C930895E4E0F0E040D0B79901C05A
:1006000030C08FEF8093680081E080936600009196
:1006100066000E3210F009F00DC0A6E6EC91FF273F
:10062000A8E691E07BE7A8D0A6E68C918F5F8C933B
:1006300008F4EDCFE2E0F0E002ED14E020E030E07D
:10064000A0E1BB2794E07BE797D0E2E2F0E001E095
:1006500010E020E030E0A0E1BB2794E07BE78CD005
:100660007CDF8CEE93E1ADE68D939C930895ED9144
:10067000FC91EF5FFF4FFC93EE93089588EE93E0BB
:1006800052D03197D9F7089522D006D000FC01D07E
:10069000089528D030D00895842F952FA62FB72FF6
:1006A0004427552766277727F1E2889409C020F46C
:1006B000480F591F6A1F7B1F769567955795479579
:1006C0003795279517950795FA9589F7089500248A
:1006D000E89477FF02C006D0689400F809D010F8BB
:1006E0000124089512D04F5F5F4F6F4F7F4F0895E1
:1006F000E89437FF089500951095209530950F5F89
:100700001F4F2F4F3F4F6894089540955095609527
:10071000709508953197F1F70895689462F80895F7
:10072000E89462F80895EF93FF93EE27E82BE92B06
:1007300031F0E8EEF3E03197F1F70197D1F7FF914F
:10074000EF91089582E001C084E099279D938A95F6
:10075000E9F70895040F151F261F371F0895041782
:100760001507260737070895E199FECFEEBB3196AE
:10077000089591E001C092E07B3751F47FB7F8947F
:10078000F3DF8D918DBBE29AE19A9A95C9F77FBF0D
:100790007727089591E001C092E0E6DFE09A8DB3FB
:0807A0008D939A95D1F708959D
:00000001FF
